:020000040800F2
:10000000001000201911000861110008611100089A
:100010006111000861110008611100080000000072
:100020000000000000000000000000006111000856
:100030006111000800000000611100086111000852
:1000400000000000000000000000000000000000B0
:1000500000000000000000000000000000000000A0
:100060000000000000000000000000000000000090
:100070000000000000000000000000000000000080
:100080000000000000000000000000000000000070
:100090000000000000000000000000000000000060
:1000A0000000000000000000000000000000000050
:1000B0000000000000000000000000000000000040
:1000C0000000000000000000000000000000000030
:1000D0000000000000000000000000000000000020
:1000E0000000000000000000000000000000000010
:1000F0000000000000000000000000000000000000
:1001000000000000000000000000000000000000EF
:1001100000000000000000000000000000000000DF
:1001200000000000000000000000000000000000CF
:1001300000000000000000000000000000000000BF
:1001400000000000000000000000000000000000AF
:10015000000000000000000000000000000000009F
:10016000000000000000000000000000000000008F
:10017000000000000000000000000000000000007F
:08018000000000000000000077
:100188000448054B10B5834203D0044B002B00D024
:10019800984710BD04000020040000200000000063
:1001A80006480749091A8910CB0F591810B5491084
:1001B80003D0044B002B00D0984710BD040000204A
:1001C800040000200000000010B5074C2378002B25
:1001D80009D1FFF7D5FF054B002B02D0044800E0FA
:1001E80000BF0123237010BD0400002000000000A0
:1001F80064110008054B10B5002B03D004490548CD
:1002080000E000BFFFF7CCFF10BDC04600000000B3
:10021800080000206411000802B47146490849002A
:10022800095C49008E4402BC7047C046002243085E
:100238008B4274D303098B425FD3030A8B4244D3A6
:10024800030B8B4228D3030C8B420DD3FF220902E8
:1002580012BA030C8B4202D31212090265D0030BA7
:100268008B4219D300E0090AC30B8B4201D3CB039D
:10027800C01A5241830B8B4201D38B03C01A5241DF
:10028800430B8B4201D34B03C01A5241030B8B42E1
:1002980001D30B03C01A5241C30A8B4201D3CB02CC
:1002A800C01A5241830A8B4201D38B02C01A5241B1
:1002B800430A8B4201D34B02C01A5241030A8B42B4
:1002C80001D30B02C01A5241CDD2C3098B4201D3CC
:1002D800CB01C01A524183098B4201D38B01C01A4A
:1002E800524143098B4201D34B01C01A52410309C1
:1002F8008B4201D30B01C01A5241C3088B4201D370
:10030800CB00C01A524183088B4201D38B00C01A1C
:10031800524143088B4201D34B00C01A5241411A43
:1003280000D20146524110467047FFE701B5002050
:1003380000F006F802BDC0460029F7D076E77047FE
:100348007047C04670B50C4D0C4E761BB61005D0E4
:10035800002408CD01349847A642FAD100F0FEFEE9
:10036800074D084E761BB61005D0002408CD013481
:100378009847A642FAD170BD9C1200089C1200084A
:100388009C120008A0120008F0B5C64600B50F2A56
:1003980043D90B00032603431E400C000300002E24
:1003A80040D11500103D2D09AC462D01A8468044CA
:1003B80000E03B00676825685F60E7681D60DF60F4
:1003C8001F00A56810379D6010344345F1D165467C
:1003D8000F230C2401352D014919134045191442E6
:1003E80023D08C59AC5104369C1B032CF9D8032418
:1003F800043B9B0801339B002240ED18C918561E88
:10040800002A07D0002300E02300CA5C5C1CEA54E1
:100418009E42F9D104BC9046F0BD0500561E002A44
:10042800F0D1F7E7561E0500ECE71A00F6E7C046DC
:10043800002382B0054A0193019B934201D902B07F
:100448007047019B01330193F6E7C046FE0F000099
:1004580010B504002078013400F052F92378002BFD
:10046800F8D110BDF8B504000E0005002B1B9E4204
:1004780004DC0023A419013C23700AE000F028F9E9
:100488002F0028700028F9D001350A28EED1002362
:100498003B70F8BD30B58DB002AC00F05DF800F0EF
:1004A80087F800F0C5F8062220492000FFF76CFF06
:1004B8001F48FFF7CDFF1F48FFF7CAFF1E48FFF789
:1004C800C7FF1E48FFF7C4FF1D48FFF7C1FF1D48BF
:1004D800FFF7BEFF1C48FFF7BBFF04AD00F0F0F8C4
:1004E8001A48FFF7B5FF20212800FFF7BBFF00F0EF
:1004F800DFF80023E15CEA5C914214D10133062B5A
:10050800F8D11348FFF7A4FF0CE0019B01330193D6
:10051800019B002BF9DDFFF78BFFFFF789FF0D48E3
:10052800FFF796FFFEE70023F1E7C04696120008A2
:1005380080110008A3110008C0110008DD1100088F
:10054800FA110008171200081A12000849120008C8
:100558007C1200086D120008F0B5902700240125D0
:100568000326042397B0FF0505A9380005930695CF
:100578000794089600F046FB102305A93800059358
:1005880006950794089600F03DFB05230AA80B93EF
:100598000A960D94139400F0C9F80723210001A8C6
:1005A800019302950394049400F0A2FA17B0F0BDE9
:1005B800802170B51B4C8902626988B00A43626168
:1005C800636990200B400193019BC023DB000393D8
:1005D80001250223032603A9C00504930595079561
:1005E800069600F00FFB8021A269C9010A43A261A7
:1005F800A3690D480B400293029B236BB3431D4331
:100608000A4B2563036096231B0243600023836023
:10061800C360036183610C33436100F06BFC08B075
:1006280070BDC04600100240240000200038014080
:1006380080201E4AF0B55169800201435161536917
:1006480087B0034090240093012500260327009BD0
:100658008023E40501A920000193029503960497DD
:1006680000F0D0FA102301A9200001930295039607
:10067800049700F0C7FA042301A92000019302950A
:100688000396049700F0BEFA32002000802100F0A3
:1006980069FB2A002000102100F064FB2A000421D5
:1006A800200000F05FFB07B0F0BDC046001002401C
:1006B800902010B501228021C00500F053FB10BD29
:1006C800902010B500228021C00500F04BFB10BD22
:1006D80037B508256B46DC1D012232232100064868
:1006E80000F03AFC002801D120783EBD034A136A85
:1006F8002B431362EEE7C046240000200038014077
:1007080007B56B46D91D0870024B0122024800F05C
:1007180099FC07BD8813000024000020024B1868CC
:10072800421C1A607047C04620000020F0B50368DC
:1007380085B00500DB072FD42B689B0700D581E027
:100748002B681B0700D5BCE02B685B0700D5DFE0F2
:100758002B68DB061AD56A69B54C0423012A00D038
:100768004BE1616B02260B436363636B1A4362635D
:10077800FFF7D4FF0700636B334200D136E1F8215D
:10078800626BAB698A43DB0013436363296A002900
:1007980000D059E1002013E00C21A54C62680A4002
:1007A800042A06D063680B40082B0BD16368DB036F
:1007B80008D523689B03BFD56B68002BBCD10120EB
:1007C80005B0F0BD6B68012B13D1802322685B0252
:1007D80013432360FFF7A2FF80260700B6022368B1
:1007E8003342A9D1FFF79AFFC01B6428F7D9032029
:1007F800E6E7002B16D123688E4A80261340236033
:1008080023688D4AB60213402360FFF787FF07006D
:100818002368334200D18FE7FFF780FFC01B6428AD
:10082800F6D9E4E7052B05D180232268DB021343C0
:100838002360CAE723687F4A1340236023687E4AFF
:100848001340C6E70C227A4C6368134206D06368EB
:100858001340082B10D16368DB030DD423689B0772
:1008680002D5EB68012BAAD1F82122682B698A43AB
:10087800DB001343236063E7EA680123002A0FD0F3
:100888002268022613432360FFF748FF0700236806
:100898003342E9D1FFF742FFC01B0228F7D9A6E788
:1008A800226802269A432260FFF738FF0700236870
:1008B800334200D144E7FFF731FFC01B0228F6D9C5
:1008C80095E7EA6901235A4C002A10D0626A022689
:1008D80013436362FFF722FF0700636A334200D0C5
:1008E80032E7FFF71BFFC01B0228F6D97FE7626AD1
:1008F80002269A436262FFF711FF0700636A3342D8
:1009080000D121E7FFF70AFFC01B0228F6D96EE7DE
:1009180080220021464C5205E3690091134208D118
:10092800E3691343E361E36913400393039B0123E2
:1009380000938027414E7F0033683B4206D0AB6866
:10094800012B13D1226A1343236230E033683B43FF
:100958003360FFF7E3FE019033683B42EFD1FFF7C6
:10096800DDFE019BC01A6428F6D940E70122002B5E
:1009780014D1236A022793432362236A03329343E1
:100988002362FFF7CBFE0600236A3B4225D0FFF720
:10099800C5FE2B4B801B9842F6D928E7052B0BD1B7
:1009A800216A013B0B432362236A1A432262FFF741
:1009B800B5FE022706000DE0236A93430422236252
:1009C800236A9343C0E7FFF7A9FE1D4B801B98429B
:1009D80000D90CE7236A3B42F5D0009B012B00D0DD
:1009E800B6E6E369174A1340E361B1E6FFF796FEFE
:1009F800C01B022800D8BEE6F9E6053203D1626BB7
:100A08009A436263BBE6626B022613430122636367
:100A1800636B93436363FFF781FE0700636B3342A5
:100A280000D1B3E6FFF77AFEC01B0228F6D9DEE64E
:100A380000100240FFFFFEFFFFFFFBFF00700040B9
:100A480088130000FFFFFFEF0C22264C012063688B
:100A58001340082B00D1B3E62368234A13402360D0
:100A680002292FD1FFF75AFE80260700B604236813
:100A7800334221D10F22E36A9343EA6A1343E362C4
:100A8800696AAB6A62680B43184980250A401343B8
:100A98006360802322685B0413432360FFF73EFEF4
:100AA8000600AD0423682B4200D073E6FFF736FE3C
:100AB800801B0228F6D99AE6FFF730FEC01B0228F1
:100AC800D5D994E6FFF72AFE80250600AD042368F1
:100AD8002B4200D15EE6FFF721FE801B0228F6D9E3
:100AE80085E6C04600100240FFFFFFFEFFFFC2FF81
:100AF800F7B501223E4C060023680F0013408B42D5
:100B080012D33268930719D4D3071FD4012322685C
:100B18001A40BA425DD833685B0761D4E122354B8D
:100B2800D2031A60002008E0236893430B43236034
:100B3800236813408B42E4D00120FEBDF0202E49EB
:100B48004B688343B06803434B60DDE72A4D726806
:100B58002B68012A1AD19B03EED503216B688B43BE
:100B680013436B60FFF7DAFD73680190012B15D111
:100B78000C226B681340042BC8D0FFF7CFFD019BF4
:100B8800C01A1E4B9842F3D90320D6E7022A02D195
:100B98009B01E2D4D0E79B07DFD4CDE7022B12D02C
:100BA8000C226B681342B1D0FFF7B8FD019BC01A45
:100BB800124B9842F4D9E7E7FFF7B0FD019BC01A42
:100BC8000E4B9842E0D80C226B681340082BF3D1E7
:100BD8009CE722689A43226022681A429BD0ABE7BE
:100BE800054A074953680B40F1680B43536095E782
:100BF800002002400000002000100240881300007E
:100C0800FFF8FFFFF0B50B6887B00393002301914D
:100C1800039ADA4001D107B0F0BD01229A4002924E
:100C28000299039A0A40009200D18CE0019A10219F
:100C3800526816008E43022E0ED107251D40AD00C6
:100C48000139A940DC08A4000419276A8F430199D7
:100C58000969A9400F43276203245F00BC40E443AD
:100C68000568013E2540AC4603251540BD40614658
:100C78000D430560012E0FD801998668CD6826407E
:100C8800BD40354385604668029915098E430121A8
:100C98000D409D4035434560C56801992C408D68DD
:100CA8008021BD4049052C43C4600A424BD0012134
:100CB800264C0326A5691E400D43A561A4699D081D
:100CC8000C400594059C0F242149AD00B6006D1811
:100CD800B4409021AF68C905A743002488420CD0CE
:100CE8001C490134884208D01B490134884204D089
:100CF8001A490134884200D00234B44000993C4378
:100D08000E00AC60164CCD4327683E43D10301D496
:100D18003E002E4026606768009E3E43910301D442
:100D28003E002E406660A768009E3E43D10201D473
:100D38003E002E40A660E668009F3743920201D429
:100D48002E403700E760013362E7C04600100240DA
:100D5800000001400004004800080048000C00485A
:100D680000040140002A01D0816170478162FCE7DC
:100D7800F8B504000E0015001F002268D36933403F
:100D88009B1B59424B41AB4201D0002018E0069B07
:100D98000133F3D0069B002B13D123680C491A6842
:100DA80003200A401A609A68A331FF318A439A6087
:100DB8002200202369321370537000236834237093
:100DC800F8BDFFF7ABFC069BC01B9842D5D9E4E7FA
:100DD8005FFEFFFF030070B59A681C69056822432F
:100DE8005C69C169224328683B4C0A43204002439E
:100DF8002A606A6839481C6A0240D86802436A60F7
:100E08009A69A8682243364C204002430320AA600E
:100E1800344A126B02403448845C802212029142A8
:100E280030D1082C2BD82000FFF7F6F90529162910
:100E38001F29292924005968E12348081B04C018E0
:100E4800FFF7F4F980B202000F2300079A43400F1E
:100E58001043E860200070BD5968244B4808C0184A
:100E6800FFF7E4F9002480B2EDE75968E123480868
:100E78001B04F4E75968802348085B02EFE7012464
:100E88000020E0E7082C24D82000FFF7C5F9052248
:100E98000E22182222221D005968E1234808DB038C
:100EA800C018FFF7C3F980B2D3E75968104B480858
:100EB800C018FFF7BBF980B2E8600024CAE7596898
:100EC800E1234808DB03F3E75968802348081B023D
:100ED800EEE70124BEE7C046F369FFFFFFCFFFFF3F
:100EE800FFF4FFFF001002407C1100080048E801F1
:100EF8000024F40070B5041E01D1012070BD050066
:100F080069352B78DBB2002B02D1020068321370EE
:100F18002423012622682B7013682000B343136032
:100F2800FFF758FFB042E8D023680A495A68002002
:100F38000A4008215A609A688A439A601A681643D8
:100F480022001E602023E0666A3268342B7013701A
:100F58002070D3E7FFF7FFFFF0B51F0003006A33E7
:100F680016001A78040085B00D000220202A39D115
:100F78000138002936D0002E34D08022A1685201D1
:100F8800914204D12269002A01D105422AD12200C6
:100F9800683211780220012924D001211170002221
:100FA800E26622321A70FFF7B9FB23008021A2689B
:100FB80058331E805E800390490104338A4215D15C
:100FC8002269002A10D11E4A1A801E8822005A322D
:100FD800108880B2002810D1230020226A33683498
:100FE8001A70207005B0F0BDFF22EDE7002AECD1A1
:100FF8002269002AF8D07F22E6E713882021013BE6
:101008009BB2138020000097039B0022FFF7B0FEDD
:10101800002813D1A268236811008022520191424E
:1010280007D12269002A04D19B8C33402B800235DA
:10103800CCE79B8C33402B700135C7E70320D1E701
:10104800FF010000F0B5070085B0039369373B78CE
:1010580004000D0016000220202B46D1013800297B
:1010680043D0002A41D08023A2685B019A4204D170
:101078002369002B01D1014237D1230068331A7844
:101088000220012A31D001221A700023E36621339D
:101098003B70FFF743FB230050331E805E808026A1
:1010A80002907601210052310A8892B2002A0DD1AD
:1010B800039B402100932000029BFFF759FE002864
:1010C80012D1202368343B7020700EE00B88002278
:1010D800013B9BB20B80039B802100932000029B65
:1010E800FFF746FE002802D0032005B0F0BDA36834
:1010F8002268B34208D12369002B05D12B88023519
:10110800DB05DB0D1385CDE72B7801351385C9E7A2
:10111800002103E00B4B5B58435004310A480B4B4A
:1011280042189A42F6D30A4A02E0002313600432B6
:10113800084B9A42F9D300E000BFFFF703F9FFF725
:10114800A9F9FEE7A412000800000020040000200E
:101158000400002094000020FEE70000F8B5C04617
:10116800F8BC08BC9E467047F8B5C046F8BC08BC39
:041178009E467047D8
:10117C00000408022A2A2A2A2A536166652D6F2D3B
:10118C006D61746963203330303020426F6F746945
:10119C006E672E2E2E0A00416C69676E696E672091
:1011AC00626974732E2E2E2E2E2E2E2E5B444F4ED5
:1011BC00455D0A00436865636B696E672043657320
:1011CC0069756D20524E472E2E5B444F4E455D0A7D
:1011DC00004D6173717565726164696E6720666C30
:1011EC006173682E2E2E5B444F4E455D0A0044659C
:1011FC006372797074696E67206461746162617383
:10120C00652E2E5B444F4E455D0A000A0A0057417D
:10121C00524E494E473A20554E415554484F52492B
:10122C005A4544204143434553532057494C4C2085
:10123C0042452050554E49534845440A00506C6570
:10124C0061736520656E7465722070617373776F5E
:10125C00726420746F20636F6E74696E75653A20CA
:10126C000050415353574F5244204641494C0A00B9
:10127C00416363657373206772616E7465642C20BF
:10128C0057656C636F6D65210A00683070783300A8
:04129C00FD01000848
:0412A000D101000870
:0412A40000127A00BA
:0400000508001119C5
:00000001FF
